:020000040000FA
:100000000002040000000000DA020000DA02000032
:10001000DA020000DA020000DA020000DA02000070
:10002000DA020000DA020000DA020000DA02000060
:10003000DA020000DA020000DA020000DA02000050
:10004000DA020000DA020000DA020000DA02000040
:10005000DA020000DA020000DA020000DA02000030
:10006000DA020000DA020000DA020000DA02000020
:10007000DA020000DA020000DA020000DA02000010
:10008000DA020000DA020000DA020000DA02000000
:10009000DA020000DA020000DA020000DA020000F0
:1000A000DA020000DA020000DA020000DA020000E0
:1000B000DA020000DA020000DA020000DA020000D0
:1000C000DA020000DA020000DA020000DA020000C0
:1000D000DA020000DA020000DA020000DA020000B0
:1000E000DA020000DA020000DA020000DA020000A0
:1000F000DA020000DA020000DA020000DA02000090
:10010000DA020000DA020000DA020000DA0200007F
:10011000DA020000DA020000DA020000DA0200006F
:10012000DA020000DA020000DA020000DA0200005F
:10013000DA020000DA020000DA020000DA0200004F
:10014000DA020000DA020000DA020000DA0200003F
:10015000DA020000DA020000DA020000DA0200002F
:10016000DA020000DA020000DA020000DA0200001F
:10017000DA020000DA020000DA020000DA0200000F
:10018000DA020000DA020000DA020000DA020000FF
:10019000DA020000DA020000DA020000DA020000EF
:1001A000DA020000DA020000DA020000DA020000DF
:1001B000DA020000DA020000DA020000DA020000CF
:1001C000DA020000DA020000DA020000DA020000BF
:1001D000DA020000DA020000DA020000DA020000AF
:1001E000DA020000DA020000DA020000DA0200009F
:1001F000DA020000DA020000DA020000DA0200008F
:10020000FFFFFF00FFFFFF00DA020000DA0200003C
:10021000DA020000DA020000DA020000DA0200006E
:10022000DA020000DA020000DA020000DA0200005E
:10023000DA020000DA020000DA020000DA0200004E
:10024000DA020000DA020000DA020000DA0200003E
:10025000DA020000DA020000DA020000DA0200002E
:10026000DA020000DA020000DA020000DA0200001E
:10027000DA020000DA020000DA020000DA0200000E
:10028000DA020000DA020000DA020000DA020000FE
:10029000DA020000DA020000DA020000DA020000EE
:1002A000DA020000DA020000DA020000DA020000DE
:1002B000DA020000DA020000DA020000DA020000CE
:1002C000DA020000DA020000DA020000DA020000BE
:1002D000DA020000DA020000DA020000DA020000AE
:1002E000DA020000DA020000DA020000DA0200009E
:1002F000DA020000DA020000DA020000DA0200008E
:10030000DA020000DA020000DA020000DA0200007D
:10031000DA020000DA020000DA020000DA0200006D
:10032000DA020000DA020000DA020000DA0200005D
:10033000DA020000DA020000DA020000DA0200004D
:10034000DA020000DA020000DA020000DA0200003D
:10035000DA020000DA020000DA020000DA0200002D
:10036000DA020000DA020000DA020000DA0200001D
:10037000DA020000DA020000DA020000DA0200000D
:10038000DA020000DA020000DA020000DA020000FD
:10039000DA020000DA020000DA020000DA020000ED
:1003A000DA020000DA020000DA020000DA020000DD
:1003B000DA020000DA020000DA020000DA020000CD
:1003C000DA020000DA020000DA020000DA020000BD
:1003D000DA020000DA020000DA020000DA020000AD
:1003E000DA020000DA020000DA020000DA0200009D
:1003F000DA020000DA020000DA020000DA0200008D
:100400000F80200080FF270000018800000000000E
:10041000050007000C000700B20202000000000007
:100420000040DA000000FE004440A9000000200067
:100430000000E0000300320000002000A00188005E
:100440004440A80000000600802D2000010020008C
:100450001600370062004000E080480091018800EB
:100460009001BA0062004000E080480091018800DD
:100470009002BA0062004000E08048000002EB00F9
:100480006028E10005003A008301E900070033001D
:10049000038009000059EB00040037006128E100E7
:1004A000010032000082EB00050007009101880086
:1004B0001001BA000200E000E6FF3A00000005006B
:1004C000910188008002780062004000E0804800CE
:1004D0003559BA008301E900080032002559BA00F5
:1004E0008301E900050032000400E000F4FF32005F
:1004F00015D9BA008301E900F1FF3A0000000600B7
:100500000400FA0010079800411020009140780084
:10051000F0CCB30000C060000044A00004E1B700CC
:1005200005E1A8000000EB00000F7800070037008D
:100530000000EB000008880001088000D01F2100A7
:10054000808F5000FCFF36001E0FE8001E00900058
:100550009E0F1000F6FF350005E1A9000080FA00AB
:10056000000006000000FA0041742000914078006D
:1005700000CEB30000C0600044E7B70044C7BF002E
:10058000F043B20044E7B70060022000303A880030
:10059000C002A900C202A900401F2000D8FF070026
:1005A000C202A800401F2000D5FF0700F9FF370056
:1005B000000000000000FE00FFFFFF00FFFFFF0043
:1005C000FFFFFF00FFFFFF00FFFFFF00FFFFFF0037
:1005D000FFFFFF00FFFFFF00FFFFFF00FFFFFF0027
:1005E000FFFFFF00FFFFFF00FFFFFF00FFFFFF0017
:1005F000FFFFFF00FFFFFF00FFFFFF00FFFFFF0007
